:020000040800F2
:1000000060230020190100089D01000895010008E7
:10001000990100088D0100089D0200080000000001
:10002000000000000000000000000000B501000812
:100030009101000800000000B1010008E50100087E
:1000400033010008330100083301000833010008C0
:1000500033010008330100083301000833010008B0
:1000600033010008330100083301000833010008A0
:100070003301000833010008330100083301000890
:100080003301000833010008330100083301000880
:100090003301000833010008330100083301000870
:1000A0003301000833010008330100083301000860
:1000B0003301000833010008330100083301000850
:1000C0003301000833010008330100083301000840
:1000D0003301000833010008330100083301000830
:1000E000330100083301000833010008000000005C
:1000F0000000000000000000000000000000000000
:1001000033010008DFF80CD000F02EF8004800475B
:10011000FD0D000860230020064880470648004780
:10012000FEE7FEE7FEE7FEE7FEE7FEE7FEE7FEE7A7
:10013000FEE7FEE7ED0100080501000830B50B46BB
:10014000014600202022012409E021FA02F59D4207
:1001500005D303FA02F5491B04FA02F52844151EDB
:10016000A2F10102F1DC30BD064C074D06E0E0686B
:1001700040F0010394E8070098471034AC42F6D3EE
:10018000FFF7C4FFE44F000804500008FEE700003A
:1001900070470000FEE70000FEE700007047000027
:1001A0004EF623510001CEF20001087070470000A6
:1001B0007047000070470000B0B501380024B4EB70
:1001C000106F1CBF0120B0BD4EF21005CEF200052D
:1001D00068600F20FFF7E4FF0720AC60286020462E
:1001E000B0BD000080B500F017F980BD80B582B0C9
:1001F00041F20000C4F20200016841F00101016017
:1002000001688907FCD5416841F080014160002107
:100210000191019A4F2A05D8019A01320192019A5F
:10022000502AF9D3426842F090024260019101994C
:100230004F2905D801990131019101995029F9D32C
:1002400041684FF6FF7221F0030141600168CFF66B
:10025000F6621140016041680C23CEF6FF0319409D
:10026000416001684FF6FF73114001600168CFF2F1
:10027000007321F4802101604168194041600168E8
:10028000114001604FF41F01816001F02DF84FF023
:100290000060002100F0EEFE02B080BDFEE700002D
:1002A000B0B543F600050446C4F200052846022115
:1002B00000F0A4FF0028F9D02846214600F078FF7E
:1002C000B0BD000010B543F60004C4F2000400BF46
:1002D0002046802100F092FF0028F9D110BD0000D7
:1002E00080B540F2026000F02DFF4FF4C06000F0D6
:1002F00029FF40F60000C4F2010028210322012357
:1003000000F0E2FC80BD000080B540F60000C4F2C1
:100310000100012100F02EFD80BD0000B0B540F2CB
:10032000036000F00FFF40F60044C4F201042046D1
:10033000102103220423042500F0C6FC6561B0BD32
:1003400040F61440C4F2010004210160704700002F
:1003500010B540F60044C4F201042046042100F028
:1003600009FDC0F10100C2B22046042100F0A6FC44
:1003700010BD0000B0B540F2026000F0E3FE40F2B4
:100380000E6000F0DFFE43F60004C4F20104A4F5A1
:1003900040552846182103224FF4007300F094FCC6
:1003A0002846042103224FF4806300F08DFC204690
:1003B00000F0F4FF20464FF4E13100F0B5FF204695
:1003C000002101F05DF82046002101F04BF82046A5
:1003D000002101F039F82046002101F02FF82046D5
:1003E000002101F025F82046042101F035F82046CF
:1003F000082101F03FF8204601F00CF8B0BD0000E4
:1004000010B5044600F08AFF044400BF00F086FFE8
:10041000A042FBD310BD000040F21C00C2F200005D
:10042000016801310160704780B540F60040C4F2B8
:1004300001004FF48051002200F040FC80BD00001C
:1004400080B540F60040C4F201004FF48051012213
:1004500000F034FC80BD000080B540F60040C4F2DE
:1004600001004FF48041002200F028FC80BD000014
:1004700080B540F60040C4F201004FF480410122F3
:1004800000F01CFC80BD000080B5FFF7B9FF80BD07
:100490002DE9F04381B08846054600200021002662
:1004A00000F084FB242000F0D7FBFFF7BDFFA5F18F
:1004B0000109002709EB0605002400BF15F8010F0C
:1004C000FFF7EEFE013C14F1FA00F7D10137102FCF
:1004D000A6EB0406EED1FFF7F5FEFFF7B1FF002013
:1004E0000021002500F062FB262000F0B5FBFFF79D
:1004F0009BFFA8F10108002608EB0504002700BFB8
:1005000014F8010F80F0FF00FFF7CAFE013F17F15A
:10051000FA00F5D10136102EA5EB0705ECD1FFF757
:10052000D1FEFFF78DFF00F05BFB01B0BDE8F0836B
:1005300010B50446102000F08FFB204600F070FB41
:1005400010BD000080B500F019FB3220FFF79CFFC2
:1005500000F020FB3220FFF797FF00F04FFB28B997
:10056000122000F079FB00F049FB08B1012080BDAA
:10057000012000F071FB272000F052FB012000F069
:100580004FFB012000F04CFB112000F065FB012027
:1005900000F046FB442000F05FFB002000F040FB31
:1005A0000F2000F03DFB452000F056FB272000F017
:1005B00037FB012000F034FB002000F031FB00206D
:1005C00000F02EFB3C2000F047FB052000F028FB4C
:1005D000212000F041FB002000F022FB802000F0F1
:1005E0001FFB182000F038FB802000F019FB4E2084
:1005F00000F032FB002000F013FB4F2000F02CFB3A
:10060000272000F00DFB012000F00AFB00F0F6FAB5
:10061000002818BF012080BDF0B587B040F202600D
:1006200000F090FD40F2036000F08CFD4FF4C060DC
:1006300000F088FD43F60004C4F2000404F55045C0
:100640002846102103224FF48073032600F03CFB60
:100650002846482103224FF4004300F035FB04F5FF
:1006600054452846102103224FF4804300F02CFB10
:100670002846182103224FF42043182700F024FBBA
:100680002846102103224FF4805300F01DFB40F256
:100690000E7000F057FD204600F08CFD6D46284698
:1006A00000F0CCFD4FF4404001904FF48270009078
:1006B00000204FF400710290CDE903102046294636
:1006C0000596069700F0A0FD204600F06BFD07B0F0
:1006D000F0BD000080B540F60000C4F201004FF408
:1006E000004100F047FB002818BF012080BD00003A
:1006F00080B540F2080CC2F2000CBCF812100029C0
:1007000008BF80BD4FF0000E06E000BFBCF812101D
:100710000EF1010E8E4512D2BCF81030002BF5D030
:100720004FF0FF31DCF800200EFB03220A4450702A
:10073000BCF810308A1C01319A42F3D3E6E780BD41
:100740002DE9F04F85B006461046B2EB060B0F467A
:10075000049248BFCBF1000BD81B80EAE07102463F
:1007600048BF4242C1EBE07904984FF0FF31B042FC
:100770004FF0FF38ABEB020A88BF4FF00108184674
:100780000293BB4288BF01210191039203E000BFA5
:10079000BBEB4A0F11DAB4B2BDB20E9A204629461D
:1007A00000F016F8B9EB4A0FF2DC049884420BD043
:1007B00003984644AAEB000AEAE70298854203D070
:1007C0000198DA440744E6E705B0BDE8F08F000081
:1007D00080B50138013980B289B200F06FF880BD70
:1007E0002DE9F04182B00F46DDE908811C4615462F
:1007F000064681B1A7420BD2B9B230462A460B4613
:10080000CDF80080FFF79CFF0137B8B2A042F3D3C8
:1008100002B0BDE8F081304639462A463B46CDF865
:100820000080FFF78DFF3046394632462346CDF82B
:100830000080FFF785FF284621462A463B46CDF833
:100840000080FFF77DFF2846214632462346CDF83B
:100850000080FFF775FF02B0BDE8F08110B540F2EF
:10086000080CDDF808E0C2F2000CCCF80000C80863
:100870004C07ACF80810ACF80A20ACF80CE04FF0CC
:10088000010E18BF0EEBD100ACF81000ACF812202E
:10089000ACF80E302BB1B42B12BF084610460A46F6
:1008A00001E010460A46ACF80400ACF8062010BD82
:1008B00040F20801C2F200010860704710B540F232
:1008C000080CC2F2000CBCF80E30B32B0BDC93B159
:1008D0005A2B36D1BCF80830C0431844BCF80A3053
:1008E000C9435C1813E0B42B0CD0B3F5877F0C46DA
:1008F00018BF10BD0BE0BCF808E0C94304460EEB7E
:10090000010004E0BCF80A30C0431C180846BCF8DB
:100910001030A4B281B26343DCF800C003EBD10E07
:100920001CF80E3000F007008024C4401C436FF018
:10093000800141FA00F0002A08BF03EA00040CF825
:100940000E4010BD2DE9F04F87B00130039080B20A
:100950000290C01AFA2800F38380082B02D10624E3
:1009600064B97DE0D8085F074FF0010618BF06EBB9
:10097000D3005F08784384B2002C71D04E1C109DC8
:10098000A2F1200041F6E44182B25808C0F600010D
:10099000DDF80C90B5FA85F70190002001EB02110B
:1009A0004FF0000804920091CDE9054312E000BF2A
:1009B00002991FFA89F0401A019926468842039845
:1009C00004BF81460836059908F101081FFA88F02E
:1009D000814245D9082B09D1049941F2486201EBC3
:1009E0004101C0F6000202EB410119E0182B0BD0C7
:1009F000102B13D00C2B33D1049941F6700201EB6C
:100A00004101C0F6000206E0049942F2D42201EB53
:100A1000C101C0F6000202EB810101E0009900BFB4
:100A2000084490F800A04FF0000B34465FEACA700B
:100A30002A461FFA89F0B1B208BF7A09FFF7C8FE4B
:100A40004FEA5A0A0136BBF1070F0BF1010BEDD348
:100A5000069B09F10109082BAAD105992646B3E79F
:100A600007B0BDE8F08F00002DE9F04F87B0DE0839
:100A70005F0705924FF0010218BF02EBD306002E6C
:100A8000009653D0119E00F1010A4A1CB6FA86F571
:100A90001FFA8AF000234FF0000B17460390CDF8A1
:100AA00010A004E00133009998B288423ED2059824
:100AB0000028F7D04FF000080293CDF804B000BF33
:100AC00010991FFA8BF00C5C4FF00009069200BFE2
:100AD000E00732461FFA8AF0B9B218BF6A09FFF779
:100AE00077FE64080137B9F1070F09F10109EFD367
:100AF0000AF1010A03991FFA8AF0401A059908F1D0
:100B000001088842049808BF8246069A1FFA88F0B6
:100B10000BF1010B08BF083288421746D0D3059865
:100B2000DDF804B0029B83441746BBE707B0BDE87D
:100B3000F08F00002DE9F04381B099461378CBB1D6
:100B4000DDF820800D4606464FEA5907541EB9F1DC
:100B5000080F08BF062700BFB0B2DAB229464B46DD
:100B6000CDF80080FFF7EEFEA3783E44002B04F1A1
:100B70000104F1D101B0BDE8F083000080B540F67A
:100B80000000C4F201004FF48071002200F096F8DA
:100B900080BD000080B540F60000C4F201004FF4B3
:100BA0008071012200F08AF880BD0000B0B50446D3
:100BB00040F22710451A4E20F92988BF2E2500F053
:100BC0004BF8C4F3C70000F02BF84F2000F044F8B6
:100BD000E8B200F025F8C5F3002000F021F8B0BD20
:100BE00080B5222000F038F8F72000F019F8202016
:100BF00000F032F800F002F880BD000010B5FFF7F9
:100C000069FD58B144F621640120013C08BF10BDC4
:100C1000FFF73AFCFFF75EFD0028F5D1002010BD7C
:100C2000B0B543F600040546C4F20004FFF7FCFB30
:100C30002046294600F0BCFA2046022100F0DEFAE8
:100C40000028F9D02046802100F0D8FA0028F9D1F8
:100C5000FFF7F6FBB0BD0000B0B543F60004054653
:100C6000C4F20004FFF7F8FBFFF7DEFB204629463D
:100C700000F09EFA2046022100F0C0FA0028F9D0C8
:100C80002046802100F0BAFA0028F9D1FFF7D8FBFE
:100C9000FFF7EEFBB0BD0000B0B543F60005C4F2AF
:100CA00001050446C1B2284600F074FB284607211E
:100CB00000F0B6FB0028F9D02046B0BD1023002A72
:100CC00008BF1423195070472DE9F047CF0601F0F3
:100CD0000F0C00F1100E00F1140A4FF000044FF059
:100CE00001094FF00F084FF0000748BF4CEA020C13
:100CF0000EE000BF166008FA04F225EA02020CFAC0
:100D000004F52A4302600137082F04F104040CD0D3
:100D100009FA07F212EA0306F5D0056828295246B7
:100D2000E8D04829E7D17246E4E7082400254FF0CF
:100D300001094FF00F080FE0176008FA05F226EAE4
:100D400002020CFA05F6324342600134102C05F120
:100D5000040508BFBDE8F08709FA04F212EA0307A8
:100D6000F3D0466828295246E6D04829E5D1724694
:100D7000E2E700008068084018BF012070470000CB
:100D8000B0B50422C4F20102134602F1180E002885
:100D900048BF73461C6800F44013B3F5401F1FFAA8
:100DA00080FC06D1156824F0706325F0706414602F
:100DB00015E0C3020AD46FF00F0303EA50430CFAA4
:100DC00003F324EA030343F0706308E0C0F3034332
:100DD000032505FA03F324EA030343F070636FF07D
:100DE0000F0404EA504400290CFA04F518BF2B4301
:100DF000002848BF72461360B0BD000088B000F004
:100E000077FA40F20020C0F2300001214FF00108D3
:100E1000FFF7B6FFFFF782FAFFF762FAFFF7AAFAC9
:100E200044F69370C0F6000000F0FCFB44F6AE7090
:100E3000C0F6000000F0F6FB44F6C670C0F60000F5
:100E400000F0F0FB44F67F70C0F6000000F0EAFB13
:100E500040F20400C2F20000016844F67070C0F66F
:100E6000000000F015FB012000F012F901465DA022
:100E700000F00EFB022000F00BF901465DA000F02F
:100E800007FB032000F004F901465EA000F000FB20
:100E900060A000F0C7FBFFF7BFFBFFF753FB40F27A
:100EA0002004C2F20004FF2620467A21FA22B4234D
:100EB0000096FFF7D3FC40F6C075C2F20005284645
:100EC0007A21FA22B4230096FFF7C8FC2046FFF7E8
:100ED000EFFCFF20FFF70CFC43F23000C0F60000EF
:100EE0000027009000200021FA227A230197FFF7C3
:100EF000BBFD2846FFF7DCFCFF20FFF7F9FB43F6BC
:100F0000D070C0F60000009000200021FA227A2361
:100F10000196FFF7A9FD20462946FFF7B9FA4FF4DD
:100F2000FA50FFF76DFA2046FFF7C2FCFF20FFF7EB
:100F3000DFFB3DA20A20002118230097FFF7FAFDEE
:100F40003EA20A201D2110230097FFF7F3FD42A2C5
:100F50000A20322110230097FFF7ECFD2846FFF707
:100F6000A7FCFF20FFF7C4FB46F26C40C0F22E0046
:100F7000069045F22070C7F26F20059046F6654056
:100F8000C6F66C70049043F63E60C4F620000390F1
:100F900003AA0A20472118230097FFF7CBFD0A2058
:100FA0006721F02274230097CDF80480FFF718FC26
:100FB00020462946FFF76CFA0120FFF7B9FA00F046
:100FC000ADF9044602E0FFF7C3F900BF00F0A6F94F
:100FD0008442FBD86434FFF797F90028F3D0FFF779
:100FE000AFF9F3E7434B5F41484220697320256422
:100FF0000D0A0000434B5F415042312069732025A8
:10100000640D0A00434B5F41504232206973202532
:10101000640D0A00457061706572204D6F64756CD7
:101020006520546573740D00322E31332045706194
:10103000706572204D6F64756C650000446573695E
:10104000676E65642042792057654163742053744C
:101050007564696F0000000077697468203235306C
:10106000207820313232207265736F6C7574696F2D
:101070006E0000004FF68072C1F6FF721140084307
:101080004EF60851CEF200010860BFF34F8F704753
:1010900010B541F20402C4F202021368014603F0E3
:1010A0000C00082841F20020C0F27A0019D1136820
:1010B00040F6001CDB03C0F23D0C03D513689B0314
:1010C00058BF844610681368C0F3834E102000EAAE
:1010D000D350704401230F2838BF0223184400FB6B
:1010E0000CF01368D2F800C0146803290DD8C3F3BC
:1010F00003130EA2D25C0FF2440E20FA02F3DFE8D3
:1011000001F01302060D184610BD002010BDCCF3EF
:1011100002201EF8000023FA00F010BDC4F3C22024
:101120001EF8000023FA00F010BD00BF0000000010
:101130000000000001020304060708090000000087
:101140000102030441F2000300F01F018009C4F210
:1011500002034FF0010CC2580CFA01F11143C150C7
:101160007047000041F2000300F01F018009C4F243
:1011700002034FF0010CC2580CFA01F122EA0101FE
:10118000C150704741F2000300F01F018009C4F212
:1011900002034FF0010CC2580CFA01F11143C15087
:1011A00070470000016841F0400101607047000095
:1011B000C160704710B543F20001C4F201018842DA
:1011C0000FD043F60041C4F2000188420CD043F630
:1011D0000001C4F20001884218BF10BD40F20E4465
:1011E00004E04FF4437401E040F20F442046FFF75F
:1011F000C9FF2046FFF7B6FF10BD00008068084019
:1012000018BF01207047000070B50268D1E902E400
:1012100002F4415CD1E90032D1E9045643EA0C03FF
:101220001A4342EA0E02224389692A433243114398
:101230000160C16921F40061C16170BD0021C0E994
:101240000511C0E90011C0E90211704741F2040024
:10125000C4F2020050F8041C41F4803140F8041C30
:101260004FF6FE7150F8043C4A1E8A4203D213F432
:1012700000311146F6D050F8041C890301D400BF98
:10128000FEE701684FF6FF7201600168CFF2C3729A
:101290000160016841F480610160016821F440311E
:1012A0000160016841F44031016001681140016052
:1012B000016841F0006141F42011016050F8041C04
:1012C00041F0807140F8041C50F8041C8901FBD5E2
:1012D000016821F003010160016841F00201016031
:1012E00001680907FCD5704780B5FFF7AFFF80BDE7
:1012F00080B540F20400C2F20000006844F6D35109
:10130000C1F26201A0FB01018809FEF755FF00B19F
:10131000FEE70520FEF744FF80BD000040F21C0000
:10132000C2F2000000687047B0B5044644F6FF30D2
:10133000C4F200000D4684424FF0000013DD44F675
:101340000041C4F200018C4219D045F20001C4F200
:1013500000018C4213D043F60001C4F201018C421B
:1013600010D103200CE044F20041C4F200018C4291
:1013700005D044F60001C4F200018C4202D10220E3
:10138000FFF786FE00EB5500B0FBF5F080B2A060E1
:10139000B0BD00006FF35F214160704710B544F6A7
:1013A000FF31C4F20001884215DD44F60041C4F269
:1013B000000188421ED045F20001C4F200018842BB
:1013C0001BD043F60001C4F20101884218BF10BDD2
:1013D00040F20E3416E044F20041C4F200018842AB
:1013E0000ED044F60001C4F20001884210D140F250
:1013F000124407E040F2134404E040F2144401E0D8
:1014000040F211442046FFF7BDFE2046FFF7AAFE3A
:1014100010BD0000C16841F40051C1607047000078
:101420008A09105801F01F01C84000F00100704700
:10143000426922F40072114341617047426922F40B
:101440008072114341617047C26822F4C062C26079
:10145000C2681143C1607047C26822F004021143A0
:10146000C1607047026922F440520261026911436F
:1014700001617047C26822F008021143C1607047E1
:10148000C26822F48052C260C2681143C1607047D2
:101490000FB4054B10B503A9044A029800F018F8E0
:1014A00010BC5DF814FB0000990C0008000000203F
:1014B00002E008C8121F08C1002AFAD1704770471D
:1014C000002001E001C1121F002AFBD1704700007B
:1014D0002DE9FF4F89B09B460446002506E02528EC
:1014E0000BD05A460B999047641C6D1C207800283D
:1014F000F5D10DB02846BDE8F08F0027B84601228F
:10150000474900E0074314F8013F203B02FA03F08B
:101510000842F7D120782E2819D114F8010F47F08E
:1015200004072A280ED06FF02F022078A0F1300196
:1015300009290CD808EB880102EB410100EB0108F6
:10154000641CF2E70A98641C50F8048B0A90207817
:101550000028CED0642808D0692806D075281ED06F
:101560005A460B9990476D1C58E00A994FF00A09AA
:1015700001C90A91002802DA40422D2102E0390512
:1015800004D52B218DF82010012103E0F90704D0A8
:101590002021F7E78A4608AE0DE00021FAE70A9914
:1015A0004FF00A0901C90A91F7E74946FEF7C6FD5F
:1015B000303106F8011D0028F7D1ADEB060000F12F
:1015C0002009780701D44FF00108C84502DDA8EBD7
:1015D000090000E000208046002706E008A85A46DF
:1015E000C05D0B9990476D1C7F1C5745F6DB04E0EE
:1015F00030205A460B9990476D1CB8F10001A8F1B4
:101600000108F5DC05E016F8010B5A460B999047E6
:101610006D1CB9F10001A9F10109F4DC641C65E756
:101620000928010010B5044601E0FFF735FB14F866
:10163000010B04490028F8D1BDE810400A20FFF74B
:101640002BBB000000000020000000000000000094
:10165000002F000000000700070000147F147F1413
:1016600000242A7F2A120062640813230036495599
:10167000225000000503000000001C224100000071
:1016800041221C000014083E08140008083E080807
:10169000000000A060000008080808080000606062
:1016A0000000002010080402003E5149453E0000A1
:1016B000427F4000004261514946002141454B3183
:1016C000001814127F10002745454539003C4A494F
:1016D00049300001710905030036494949360006C1
:1016E0004949291E00003636000000005636000029
:1016F00000081422410000141414141400004122A4
:10170000140800020151090600324959513E007C7B
:101710001211127C007F49494936003E4141412265
:10172000007F4141221C007F49494941007F09094E
:101730000901003E4149497A007F0808087F0000FE
:10174000417F4100002040413F01007F08142241B9
:10175000007F40404040007F020C027F007F040871
:10176000107F003E4141413E007F09090906003ECD
:101770004151215E007F09192946004649494931F6
:101780000001017F0101003F4040403F001F204019
:10179000201F003F4038403F0063140814630007D7
:1017A0000870080700615149454300007F4141002E
:1017B00000552A552A55000041417F0000040201CE
:1017C00002040040404040400000010204000020AC
:1017D00054545478007F48444438003844444420EA
:1017E00000384444487F00385454541800087E0997
:1017F00001020018A4A4A47C007F0804047800005F
:10180000447D4000004080847D00007F102844001B
:101810000000417F4000007C04180478007C08042C
:10182000047800384444443800FC24242418001868
:10183000242418FC007C0804040800485454542054
:1018400000043F444020003C4040207C001C2040DD
:10185000201C003C4030403C004428102844001C20
:10186000A0A0A07C004464544C4414141414141418
:101870000000000000000000000000000000FC006C
:101880000000000002000000000C020C020000003A
:101890000000000090D0BCD0BC900003000300000A
:1018A0001824FE448C000302070201001824D8B05B
:1018B0004C80000300010201C038E438E00001025E
:1018C0000201020208060000000000000000000003
:1018D000000000F80402000000010204000204F805
:1018E00000000004020100009060F8609000000019
:1018F000010000002020FC2020000000010000006A
:101900000000000000000806000000002020202049
:1019100020000000000000000000000000000002A5
:10192000000000000080601C0200040300000000B2
:10193000F8040404F8000102020201000008FC009F
:10194000000000020302000018844424180003026F
:101950000202020008042424D8000102020201004D
:1019600040B088FC80000000000302003C242424D6
:10197000C400010202020100F824242CC00001026C
:10198000020201000C04E41C04000000030000003B
:10199000D8242424D800010202020100384444441F
:1019A000F800000302020100000010000000000027
:1019B00002000000000020000000000006000000FF
:1019C00000205088040200000000010290909090D6
:1019D0009000000000000000000204885020000277
:1019E000010000001804C4241800000002000000D8
:1019F000F804E494F80001020202020000E09CF006
:101A0000800002030000030204FC2424D800020327
:101A100002020100F80404040C00010202020100A9
:101A200004FC0404F80002030202010004FC247414
:101A30000C0002030202030004FC24740C000203E5
:101A400002000000F0080444CC4000010202010042
:101A500004FC2020FC040203000003020404FC0434
:101A60000400020203020200000404FC0404060451
:101A70000403000004FC24D00C040203020003024F
:101A800004FC04000000020302020203FC3CC03C10
:101A9000FC0003000300030004FC30C4FC04020348
:101AA00002000300F8040404F8000102020201002D
:101AB00004FC24241800020302000000F8848404BB
:101AC000F80001020207050004FC246498000203E8
:101AD00002000302182424448C00030202020100C5
:101AE0000C04FC040C0000020302000004FC0000D3
:101AF000FC04000102020100047C80E01C040000E0
:101B0000030000001CE03CE01C0000030003000098
:101B1000049C609C0400020300030200041CE01CFF
:101B200004000002030200000C84641C0400020391
:101B3000020203000000FE0202000000070404008D
:101B4000000E30C00000000000010200000202FE92
:101B5000000000040407000000040204000000006C
:101B60000000000000000000000008080808080845
:101B70000000020000000000000000000040A0A0E3
:101B8000C00000010202030204FC2020C000000388
:101B90000202010000C020206000000102020200D9
:101BA00000C02024FC0000010202030200C0A0A02B
:101BB000C0000001020202000020F82424040002F8
:101BC000030202000040A0A0602000070A0A0A04E5
:101BD00004FC2020C0000203020003020020E400F5
:101BE0000000000203020000000020E400000808DA
:101BF0000807000004FC80E020200203020003022A
:101C00000404FC000000020203020200E020E020C5
:101C1000C00003000300030020E02020C0000203F6
:101C20000200030200C02020C000000102020100E7
:101C300020E02020C000080F0A02010000C0202080
:101C4000E0000001020A0F0820E04020200002030B
:101C5000020000000060A0A02000000202020300B9
:101C60000020F820000000000102020020E0002017
:101C7000E00000010202030220E02080602000005A
:101C8000030100006080E0806000000300030000AA
:101C900020608060200002030003020020E020801A
:101CA00060200808070100000020A060200000025A
:101CB00003020200000020DE020000000007040012
:101CC000000000FF00000000000F00000002DE2006
:101CD00000000004070000000201020404020000EA
:101CE00000000000000000000000000000000000F4
:101CF00000000000000000F80000000000000033B9
:101D00003000000000100C06100C0600000000005F
:101D10000000000040C07840C0784000043F040448
:101D20003F040400007088FC08300000001820FF09
:101D3000211E0000F008F000E018000000211C0344
:101D40001E211E0000F00888700000001E212324C0
:101D50001927211010160E000000000000000000DE
:101D600000000000000000E018040200000000076E
:101D70001820400000020418E00000000040201875
:101D800007000000404080F0804040000202010F48
:101D900001020200000000F0000000000101011F2C
:101DA00001010100000000000000000080B0700090
:101DB0000000000000000000000000000001010120
:101DC00001010101000000000000000000303000AF
:101DD0000000000000000000806018040060180689
:101DE0000100000000E010080810E000000F1020C3
:101DF00020100F00001010F8000000000020203F0D
:101E00002020000000700808088870000030282496
:101E10002221300000300888884830000018202037
:101E200020110E000000C02010F80000000704245C
:101E3000243F240000F808888808080000192120A1
:101E400020110E0000E0108888180000000F1120FB
:101E500020110E0000380808C83808000000003FB4
:101E6000000000000070880808887000001C222113
:101E700021221C0000E010080810E00000003122C0
:101E800022110F00000000C0C00000000000003060
:101E900030000000000000800000000000008060B2
:101EA0000000000000008040201008000001020433
:101EB000081020004040404040404000040404041A
:101EC00004040400000810204080000000201008D6
:101ED00004020100007048080808F000000000300B
:101EE00036010000C030C828E810E0000718272499
:101EF00023140B000000C038E0000000203C230247
:101F00000227382008F8888888700000203F2020A9
:101F100020110E00C03008080808380007182020DB
:101F20002010080008F808080810E000203F2020D2
:101F300020100F0008F88888E8081000203F2020B3
:101F40002320180008F88888E8081000203F2000A7
:101F500003000000C03008080838000007182020DF
:101F6000221E020008F808000008F808203F21019E
:101F700001213F20000808F8080800000020203F49
:101F80002020000000000808F8080800C0808080B9
:101F90007F00000008F888C028180800203F2001B2
:101FA0002638200008F8080000000000203F20200C
:101FB0002020300008F8F800F8F80800203F003F23
:101FC000003F200008F830C00008F808203F20003B
:101FD00007183F00E01008080810E0000F1020204C
:101FE00020100F0008F808080808F000203F210121
:101FF00001010000E01008080810E0000F18242478
:1020000038504F0008F8888888887000203F2000EA
:10201000030C3020007088080808380000382021A0
:1020200021221C00180808F8080818000000203FAA
:102030002000000008F808000008F808001F202011
:1020400020201F000878880000C8380800000738E2
:102050000E010000F80800F80008F800033C070033
:10206000073C0300081868808068180820302C039B
:10207000032C30200838C800C83808000000203F72
:102080002000000010080808C83808002038262161
:1020900020201800000000FE020202000000007F65
:1020A00040404000000C30C0000000000000000173
:1020B0000638C00000020202FE000000004040405E
:1020C0007F00000000000402020204000000000083
:1020D0000000000000000000000000008080808000
:1020E00080808080000202040000000000000000E8
:1020F0000000000000008080808000000019242281
:1021000022223F2008F8008080000000003F1120BC
:1021100020110E000000008080800000000E1120C1
:1021200020201100000000808088F800000E11209F
:1021300020103F200000808080800000001F2222AD
:1021400022221300008080F0888888180020203F19
:10215000202000000000808080808000006B94942C
:102160009493600008F8008080800000203F2100E8
:1021700000203F2000809898000000000020203FB1
:1021800020200000000000809898000000C080809F
:10219000807F000008F8000080808000203F24023B
:1021A0002D302000000808F8000000000020203F2B
:1021B000202000008080808080808000203F2000E0
:1021C0003F20003F8080008080800000203F210071
:1021D00000203F200000808080800000001F202021
:1021E00020201F00808000808000000080FFA12050
:1021F00020110E000000008080808000000E112061
:1022000020A0FF80808080008080800020203F21EF
:1022100020000100000080808080800000332424A2
:1022200024241900008080E0808000000000001F4E
:10223000202000008080000000808000001F2020FF
:1022400020103F20808080000080808000010E30C0
:102250000806010080800080008080800F300C0321
:102260000C300F0000808000808080000020312E24
:102270000E312000808080000080808080818E7000
:102280001806010000808080808080000021302CB2
:102290002221300000000000807C020200000000CB
:1022A000003F404000000000FF0000000000000070
:1022B000FF0000000002027C800000000040403F60
:1022C00000000000000601010202040400000000FA
:1022D00000000000000000000000000000000000FE
:1022E00000000000000000000000000000000000EE
:1022F00000000000000000000000000000F0F0F00E
:10230000000000000000000000017F01000000004C
:1023100000000000001C1C1C000000000000806089
:10232000301C8C60301C0C0000000000000000001D
:10233000000000000000000000000000000000009D
:10234000000000E00000000000E000000086E69FC2
:1023500086868686E69F860000011F010101010135
:102360001F010100000080C06020F820E0C00000D4
:10237000000003070C18FF70E18100000000070F48
:1023800010107F100F0700008060206080000000A8
:10239000E02000000F3020309F70DC371030C0008C
:1023A0000000100E03000718101807000000C020DE
:1023B00020E0C0000000000080E01F38E88703C470
:1023C0003C040000070F1810100B070D1010080038
:1023D00000808C4C3800000000000000000000006D
:1023E00000000000000000000000000000000000ED
:1023F0000000000000000000000080E03008040041
:102400000000000000FEFF010000000000000000CE
:102410000000030F1820400000040830E080000096
:10242000000000000000000001FFFE0000000000AE
:10243000004020180F030000000000000000000012
:102440000000C00000000000004266663C18FF1853
:102450003C6666420000000000000300000000002F
:1024600000000000000080000000000000101010BC
:102470001010FF10101010100000000000000300EA
:10248000000000000000000000000000000000004C
:1024900000000000000000000000000000808C4CE4
:1024A00038000000000000000000000000000000F4
:1024B000000000000010101010101010101010007C
:1024C000000000000000000000000000000000000C
:1024D00000000000000000000000000000000000FC
:1024E0000000000000001C1C1C0000000000000098
:1024F0000000000000000000E0380C0000000000B8
:1025000080701C03000000000060380E0100000015
:1025100000000000000080C060202060C08000003B
:1025200000FEFF010000000001FFFE000001070E99
:10253000181010180E0701000000808080C0E00015
:10254000000000000000000000FFFF00000000008D
:1025500000001010101F1F101010000000804020FD
:1025600020202060C080000000030300804020384D
:102570001F070000001C1A1918181818181F00004F
:102580000080C020202060C0800000000003030005
:102590001010182FE780000000070F1010101018FF
:1025A0000F070000000000000000C0E0F000000085
:1025B00000C0B088868180FFFF808000000000009E
:1025C0000010101F1F1010000000E06060606060CD
:1025D0006060000000003F1008080818F0E00000EC
:1025E00000070B101010101C0F030000000080C02B
:1025F00040202020E0C0000000FCFF211008080857
:1026000018F0E0000001070C18101010080F03006C
:102610000000C0E06060606060E0600000000300F7
:102620000000E0180700000000000000001F1F006D
:10263000000000000080C0602020202060C08000DA
:102640000087EF2C1818303068CF830000070F0880
:1026500010101010180F07000000C0C0202020200C
:10266000C0800000001F3F604040402010FFFE007F
:1026700000000C1C101010080F03000000000000E8
:10268000000000000000000000000000000E0E0E20
:102690000000000000000000001C1C1C00000000E6
:1026A000000000000000000000000000000000002A
:1026B000000C0C0000000000000000000058380072
:1026C000000000000000000000000080402010001A
:1026D00000001028448201000000000000000000FB
:1026E00000000102040810000000000000000000CB
:1026F00000000000008484848484848484848400B2
:102700000000000000000000000000000000102099
:102710004080000000000000000000000000018276
:10272000442810000000100804020100000000000E
:1027300000C020201010101030E0C0000003030083
:1027400000F010080C070300000000001C1C1C0017
:1027500000000000000000C0406020202040C000B9
:1027600000FCFF01F00E03C1FE03807F0001070E95
:1027700008111110110904020000000080E0E000BF
:10278000000000000000807C4340477FF88000008C
:1027900010181F1000000000131F1C1020E0E02084
:1027A00020202060C080000000FFFF1010101018D3
:1027B0002FE78000101F1F1010101010180F0700B7
:1027C000000080C0402020202060E00000FCFF01CD
:1027D00000000000000001000001070E181010109A
:1027E0000804030020E0E02020202040C0800000FA
:1027F00000FFFF000000000001FFFE00101F1F107F
:10280000101018080E07010020E0E02020202020F2
:102810002060800000FFFF101010107C00000000FE
:10282000101F1F10101010101018060020E0E020DC
:10283000202020206060800000FFFF101010107C1E
:1028400000000100101F1F10000000000000000029
:10285000000080C06020202040E0000000FCFF015C
:1028600000004040C0C140400001070E1810101089
:102870000F0F000020E0E0200000000020E0E0203A
:1028800000FFFF101010101010FFFF00101F1F108E
:1028900000000000101F1F100000202020E0E0209A
:1028A000202000000000000000FFFF0000000000EA
:1028B00000001010101F1F1010100000000000007A
:1028C000202020E0E020202000000000000000FF89
:1028D000FF0000000060E0808080C07F3F000000BB
:1028E00020E0E020000020A06020200000FFFF305A
:1028F000187CE3C000000000101F1F10000001132F
:102900001F1C181020E0E020000000000000000064
:1029100000FFFF000000000000000000101F1F105B
:10292000101010101018060020E0E0E00000000079
:10293000E0E0E02000FF013FFEC0E01E01FFFF00DD
:10294000101F1000031F0300101F1F1020E0E0C025
:10295000000000000020E02000FF0003071C78E0DA
:102960008000FF00101F100000000000030F1F0078
:10297000000080C060202060C080000000FEFF01D9
:102980000000000000FFFE000001070E18101018E4
:102990000C07010020E0E0202020202060C0800003
:1029A00000FFFF2020202020301F0F00101F1F10CD
:1029B0000000000000000000000080C060202060D7
:1029C000C080000000FEFF010000000000FFFE00CC
:1029D0000001070E1111133C7C67210020E0E0206C
:1029E0002020202060C0800000FFFF101030F0D0B9
:1029F000080F0700101F1F10000000030F1C10100D
:102A00000080C060202020204040E00000070F0C24
:102A10001818303060E08100001F0C0810101010F2
:102A2000180F07008060202020E0E0202020608038
:102A30000100000000FFFF00000000010000000096
:102A4000101F1F100000000020E0E0200000000028
:102A50000020E02000FFFF00000000000000FF0059
:102A600000070F1810101010100807002060E0E099
:102A70002000000020E060200000077FF880008038
:102A80007C03000000000000071F1C07000000007E
:102A900020E0E02000E0E0200020E0200007FFF838
:102AA000E01FFFFCE01F00000000031F0300011FE8
:102AB00003000000002060E0A0000020E060200093
:102AC000000000038F7CF8C6010000000010181EF3
:102AD000130001171F1810002060E0E02000000024
:102AE00020E06020000001073EF8E0180700000029
:102AF00000000010101F1F10100000000080602058
:102B0000202020A0E0E0200000000000C0F03E0FE8
:102B10000300000000101C1F1710101010180600F2
:102B20000000000000FC0404040404000000000095
:102B300000FF00000000000000000000007F404097
:102B400040404000000010E00000000000000000D5
:102B500000000000031C6080000000000000000076
:102B6000000000030C70800000000404040404FC56
:102B70000000000000000000000000FF0000000056
:102B8000000040404040407F000000000000001076
:102B9000080C040C081000000000000000000000F9
:102BA0000000000000000000000000000000000025
:102BB0000000000000000000000000000000000015
:102BC0000000000000000000808080808080808005
:102BD00080808080000000040408080000000000DD
:102BE00000000000000000000000000000000000E5
:102BF00000000000000000000000000000000000D5
:102C000000000000000098D844642424FCF8000070
:102C1000000F1F18101010081F1F10180020E0F0E0
:102C200000000000000000000000FFFF180804047E
:102C30000CF8F00000001F0F18101010180F030000
:102C400000000000000000000000000000E0F81894
:102C50000404043C3800000000030F0C1010101096
:102C6000080600000000000000000020E0F0000066
:102C700000E0F81C04040408FFFF000000030F1824
:102C8000101010081F0F08000000000000000000D6
:102C9000000000000000E0F8484444444C78700014
:102CA0000000030F0C1810101008040000000000B2
:102CB00080C0602020E0C00000040404FFFF040482
:102CC00004040000000010101F1F1010100000006E
:102CD000000000000000000000000000000070F88C
:102CE0008C04048CF874040C007076CF8D8D8D8963
:102CF000C87870000020E0F0000000000000000034
:102D00000000FFFF08040404FCF8000000101F1F6F
:102D1000100000101F1F1000000000000060600085
:102D2000000000000000040404FCFC00000000009F
:102D300000001010101F1F101010000000000000F5
:102D4000000000606000000000000000040404FCBB
:102D5000FC0000000000C0C08080C07F3F00000079
:102D60000020E0F000000000000000000000FFFF75
:102D700080C0F41C0404000000101F1F1100031F7A
:102D80001C1010000000202020E0F00000000000D7
:102D90000000000000FFFF00000000000000101015
:102DA000101F1F10101000000000000000000000A5
:102DB0000000000004FCFC0804FCFC0804FCFC000F
:102DC000101F1F10001F1F10001F1F100000000009
:102DD00000000000000000000004FCFC08080404DF
:102DE000FCF8000000101F1F100000101F1F100033
:102DF00000000000000000000000000000E0F018EB
:102E00000C04040C18F0E00000030F0C101010105C
:102E10000C0F030000000000000000000000000094
:102E20000004FCFC080404040CF8F0000080FFFF20
:102E3000889010101C0F030000000000000000002C
:102E40000000000000E0F81C04040408F8FC000086
:102E500000030F1810109088FFFF80000000000092
:102E60000000000000000000040404FCFC10080442
:102E7000040C0C001010101F1F1010100000000098
:102E8000000000000000000000000000000030789A
:102E9000CCC48484840C1C0000001E181010101177
:102EA000190F06000000000000C000000000000034
:102EB00000040404FFFF04040400000000000000FC
:102EC0000F1F1010100C0000000000000000000098
:102ED000000000000004FCFE00000004FCFE0000F6
:102EE00000000F1F181010081F0F0800000000003E
:102EF000000000000000000000040C3CFCC40000C6
:102F0000C43C0C0400000000010F1E0E0100000074
:102F1000000000000000000000000000043CFCC4B1
:102F200000E47CFC84807C040000071F070000078D
:102F30001F0700000000000000000000000000006B
:102F40000004041C7CE4C0341C0404000010101CA9
:102F50001601131F1C1810000000000000000000E4
:102F60000000000000040C3CFCC400C43C0404004D
:102F70000000C080C1370E0100000000000000000A
:102F8000000000000000000000001C0404C4F47CE9
:102F90001C0400000000101C1F17111010180E0058
:102FA00000000000000000F80C0400000000000019
:102FB000001028EF00000000000000000000003FAB
:102FC00060400000000000000000FF000000000062
:102FD000000000000000FF000000000000000000F2
:102FE0000000FF00000000000000040CF8000000DA
:102FF0000000000000000000EF28100000000000AA
:10300000000040603F0000000000000000180602C1
:10301000020408102020300800000000000000001A
:1030200000000000000000000000000000000000A0
:103030000000000000000000000000000000000090
:103040000000000000000000000000000000000080
:103050000000000000000000000000000000000070
:1035D00000000000000000008080808080800000EB
:1035E000000000C0E0E0E0E0C0C00000000000001B
:1035F00000000000000000000000000000000000CB
:1036000000000000000000000000000000000000BA
:10361000000000000000000000007EFEFEFEFEFE36
:10362000FE00000080FEFEFEFEFEFEFEFC0000002E
:1036300000FCFEFEFEFEFE3E00000000000000005A
:10364000808080808080000000000000000000007A
:10365000000080F8FEFEFEFEFEFEFEFEF080000092
:1036600000000000000000000000008080808080DA
:1036700080000000000000F8F8F8F8F8F8F8000002
:103680000000000000000000000000000000E0F06A
:10369000F8FCFCFEFE7E7E3E3E7E7EFEFCFC78302C
:1036A00000000000F8F8F8F8F8F8F8000000000052
:1036B000000000000000000000000000000000000A
:1036C00000000000000000000000000080808080FA
:1036D0008000FFFFFFFFFFFFFF000000030F1F1F21
:1036E0001F1F0F0F000000000000000000808080FE
:1036F00080808080000000000000000000000000CA
:1037000000000000000000000000000000000000B9
:1037100000000000003FFFFFFFFFFFFC00C0FFFFB5
:10372000FFFF7FFFFFFFFFFF8000FEFFFFFFFFFFA8
:103730000F000000F0F8FEFEFFFF7F1F0F0F1FFFBE
:10374000FFFFFEFCF8C000000000C0FCFFFFFFFF11
:103750007F071FFFFFFFFFFFF88000000000C0F0A1
:10376000FCFEFFFFFF7F1F1F1F1F3F3F3F0E041F79
:103770001FFFFFFFFFFFFFFF1F1F1F1F00000000B5
:1037800000000000000000001F7FFFFFFFFFFFFCA4
:10379000F8F8F0F0E0E0C1C08000001F1F1FFFFF3D
:1037A000FFFFFFFFFF1F1F1F0F000000FFFFFFFFB6
:1037B000FFFF00000000FFFFFFFFFFFFFF00000012
:1037C000C0F8FCFEFFFFFF7F1F1F1F3FFFFFFFFF33
:1037D000FFFFFF00000000FFFFFFFFFFFFFF0000F3
:1037E00000C0F8FCFEFFFFFF3F1F1F1F3FFFFFFF52
:1037F000FEFCF8E0000000000000000000000000F7
:1038000000000000000000000000000000000000B8
:103810000FFFFFFFFFFFFCFFFFFFFF1F0001FFFF88
:10382000FFFFFFFEFFFFFFFFFF070000001EFFFF7F
:10383000FFFFFFFFDF1F1F1F1F1F1F9F9F1F1F1F58
:103840000000E0FEFFFFFFFFFFFFFCFCFCFDFFFFB1
:10385000FFFFFFFFFCC00000FFFFFFFFFFFFFF8037
:103860000000000000800000000000FFFFFFFFFFDD
:10387000FFFF00000000000000000000000000004A
:10388000000080C0C0800101030303070FFFFFFF9A
:10389000FFFFFFFF70000000FFFFFFFFFFFFFF00C3
:1038A000000000000000FFFFFFFFFFFF000000809E
:1038B000FFFFFFFFFFFFFF000000FFFFFFFFFFFF15
:1038C000FF8000000000FFFFFFFFFFFFFF00000080
:1038D00000FFFFFFFFFFFFFF000000FFFFFFFFFFF4
:1038E000FFFF8000000000FFFFFFFFFFFFFF000061
:1038F00000000000000000000000000000000000C8
:103900000000000000000000000000073F3F3F3FB4
:103910003F3F3F3F0F000000003F3F3F3F3F3F3FE3
:103920003F3F01000000000001070F1F1F3F3F3F06
:103930003E3E3E3E3F3F1F1F0E00303E3F3F3F3F5B
:103940003F1F01000000000000033F3F3F3F3F3F9B
:103950003C000003070F1F3F3F3F3F3E3E3F3F3FBE
:103960001F1E080000030F1F3F3F3F3F3F3E3F3FEA
:103970001C18000000000000000000070F1F1F3F80
:103980003F3F3F3E3E3F3F3F3F1F1F0F07030000AB
:103990000000070F1F3F3F3F3F3E3F3F3F1C0000DF
:1039A0000F1F3F3F3F3F3F3E3F1F1F3F3F3F3F3FB8
:1039B0003F00000000070F1F3F3F3F3F3F3E3F1FBC
:1039C0001F3F3F3F3F3F3F000000003F3F3F3F3F23
:1039D0003F3F0000000003070F1F3F3F3F3F3E3EB9
:1039E0003F3F3F1F1F0F03000000000000000000CA
:1039F00000000000000000000000000000000000C7
:103A000000000000000000000000000000000000B6
:103A100000000000000000000000000000000000A6
:103A20000000000000000000000000000000000096
:10410000C0C0C0C0C0000080C0C0C0C080000000EF
:10411000000000000000000000000000000000009F
:10412000000000000000000000000000000000008F
:10413000000000000000000000000000000000007F
:10414000000000000000000000000000000000006F
:10415000000000000000000000000000000000005F
:10416000000000000000000000000000000000004F
:10417000000000000000000000000000000000003F
:10418000000000000000000000000000000000002F
:10419000000000C0C0C0C0C0C0000000000000009F
:1041A000000000000000000000C0C0C0C0C000004F
:1041B00000000000000000000000000000000000FF
:1041C000000000000000000000000000000C1E1FA6
:1041D0001F0F0F9FFFFFFEFEF80000000000000011
:1041E00038787C7E3EFFFFFFFFFF00040E1E1F8F0E
:1041F0008F8FFFFFFFFEFC000000737F3F1F0F004B
:1042000000317B7F3F1F070000000000000000FF1F
:10421000FFFFFFFF8787878787070000F0F0F0F038
:10422000F0F070F8F8F0F0E0800030F0F0F078781E
:10423000F8F0F0F0E0800000F0F0F0F0F0F070F84E
:10424000F8F0F0E0800080E0F0F0F0F878F0F0F0C6
:10425000E0C00000F0F0F0F0F0F0F0F0F01000003E
:104260000000000000FFFFFFFFFFFFFEC0E0FFFFB8
:10427000FFFFFFFFFF000080C0E0F0F0F078F8F0F3
:10428000F0F0E0C00000C0E0F0F0F8F870FFFFFFD1
:10429000FFFFFF0000F0F0F0F0F000F0F0F0F0F0C1
:1042A000F00000FFFFFFFFFF000080C0E0F0F0F82B
:1042B00078F8F0F0F0E0800000000000000000005E
:1042C0000000000000000080C0F0F8FCFEFFBF9F6F
:1042D00087838000C0C0C0C0C0800000000000FF15
:1042E000FFFFFFFF0080C0C0C0C78787CFFFFFFF71
:1042F000FEF80000000000000000000000000000C8
:10430000000000000000000000FFFFFFFFFF8787A4
:10431000878787800000FFFFFFFFFF8080E1FFFFAE
:10432000FFFF7F40F8FCFCFEFE9ECFFFFFFFFFFF7C
:104330000000FFFFFFFFFF8080E1FFFFFFFF7F0026
:10434000FFFFFFFFFFDC9C9D9FDFDF9F1F00FFFF44
:10435000FFFFFF0301000000000000000000FFFF5E
:10436000FFFFFF0FFFFFFFFFFFFF0FFFFFFFFFFC40
:10437000007FFFFFFFFFE18080FFFFFFFFFF1C08C2
:10438000FFFFFFFFFF8080FFFFFFFFFFFF0000FF39
:10439000FFFFFFFF80FFFFFFFFFFFF0000FFFFFFAA
:1043A000FFFF80007FFFFFFFFFDC9C9C9FDFDF9F04
:1043B0001F000000000000000000000000000000DE
:1043C000000707070707070707070707070003078F
:1043D00007070703000000000007070707070001A1
:1043E0000303070707070707070301000000000092
:1043F00000000000000000000000000000000000BD
:10440000000000070707070707070707070700005F
:10441000FFFFFFFFFF070707070703010000030770
:10442000070707070703070707070000FFFFFFFF4E
:10443000FF0707070707030100000001030707073D
:104440000707070703030000070707070700000027
:104450000000000000000000070707070700010137
:104460000101010000070707070700000103070714
:1044700007070707070303000000010307070707F3
:1044800007070707070707000003070707070707CE
:1044900007070707070000030707070707070001CB
:1044A00003070707070707070303000000000000D2
:1044B00000000000000000000000000000000000FC
:1044C00000000000000000000000000000000000EC
:1044D00000000000000000000000000000000000DC
:1044E00000000000000000000000000000000000CC
:104AC0000000000070F0F8FC7CFEFEFEFEFE001808
:104AD0003C3C3E3E1E1EFEFEFEFCF800183C3E3EE8
:104AE0001E1E3EFEFEFCFCF000000000000000E088
:104AF000E0E0E0E0C080E0E0E0E0E0000000000096
:104B000000183C3C3E3E1E1EFEFEFEFCF80000FE71
:104B1000FEFEFEFE9E9E9E9E1E1E0000E0F8FCFE17
:104B2000FE7E1E3EFEFEFCF8E000000000000000DD
:104B300000FEFEFEFEFEFE0E0E0E0E0E0E0000002D
:104B4000000000000000000000FEFEFEFEFE00006F
:104B50000000000000FEFEFEFEFE000000FEFEFE65
:104B6000FEFEFEFCE000FEFEFEFEFE0000FEFEFE7F
:104B7000FEFEC0E0F8FCFEFE3E1E06000000000047
:104B80000000000000000000000000000000000025
:104B90000000000000000000000000000000000015
:104BA0000000000000000000000000000000000005
:104BB00000000000000000000000000000000000F5
:104BC000000000FFFFFFFFFF000080C0E0F0FCFEE0
:104BD0007F3F1F0F03000080E0F0F8FCFF7F3F0FD6
:104BE00007010000000000000000C1E7FFFFFFFF19
:104BF000FFFFF7C1000000000000000080C0E0F0EF
:104C0000FCFE7F3F1F0F0300008787878707078F02
:104C1000FFFFFFFFFC007FFFFFFFFFC00080FFFFE3
:104C2000FFFFFF0000000000000000FFFFFFFFFF8C
:104C3000FF0F0F0F0F0F00001E1E1E1E1E1E1E1E3A
:104C40001E0000FFFFFFFFFF00000000000000FF4C
:104C5000FFFFFFFF000000FFFFFFFFFF3FFFFFFF21
:104C6000FFFFFFFFFF0000FFFFFFFFFF1F7FFFFFB2
:104C7000FFF8E0C00000000000000000000000009D
:104C80000000000000000000000000000000000024
:104C90000000000000000000000000000000000014
:104CA0000000000000000000000000000000000004
:104CB000000000000000000000000000000F0F0FC7
:104CC0000F0F00000F0F0F0F0F0F0F0F0F0F0F071A
:104CD0000F0F0F0F0F0F0F0F0F0F0F0F0000000020
:104CE00000000C0F0F0F0F0F0101070F0F0F0F0C1C
:104CF0000000000000000F0F0F0F0F0F0F0F0F0F1E
:104D00000F070307070F0F0F0F0F0F0F0703010008
:104D10000003070F0F0F0F0F0F0F07030000000016
:104D200000000000000F0F0F0F0F0F0F0F0F0F0FDE
:104D30000F0000000000000000000000000F0F0F37
:104D40000F0F0F0F0F0F0F0F000F0F0F0F0F0000A0
:104D5000000F0F0F0F0F00010F0F0F0F0F0F0F009E
:104D6000000F0F0F0F0F000001030F0F0F0F0F0C9D
:104D70000000000000000000000000000000000033
:104D80000000000000000000000000000000000023
:104D90000000000000000000000000000000000013
:104DA0000000000000000000000000000000000003
:104DB00000000000000000000000000000000000F3
:104DC00000000000000000000000000000000000E3
:104DD00000000000000000000000000000000000D3
:104DE00000000000000000000000000000000000C3
:104DF00000000000000000000000000000000000B3
:104E000000000000000000000000000000000000A2
:104E10000000000000000000000000000000000092
:104E20000000000000000000000000000000000082
:104E30000000000000000000000000000000000072
:104E40000000000000000000000000000000000062
:104E50000000000000000000000000000000000052
:104E60000000000000000000000000000000000042
:104E70000000000000000000000000000000000032
:104E80000000000000000000000000000000000022
:104E90000000000000000000000000000000000012
:104EA0000000000000000000000000000000000002
:104EB00000000000000000000000000000000000F2
:104EC00000000000000000000000000000000000E2
:104ED00000000000000000000000000000000000D2
:104EE00000000000000000000000000000000000C2
:104EF00000000000000000000000000000000000B2
:104F000000000000000000000000000000000000A1
:104F10000000000000000000000000000000000091
:104F20000000000000000000000000000000000081
:104F30000000000000000000000000000000000071
:104F40000000000000000000000000000000000061
:104F50000000000000000000000000000000000051
:104F60000000000000000000000000000000000041
:104F700053797374656D436C6B3A25640D0A007741
:104F80007777772E77656163742D74632E636E0D6A
:104F90000A0D000D0A5765416374205374756469E6
:104FA0006F20436F726520426F6172640D007765F8
:104FB00061637473747564696F2E74616F62616F7D
:104FC0002E636F6D0D00776561637473747564692A
:104FD0006F2E616C69657870726573732E636F6D87
:104FE0000D0000000850000800000020080000002C
:104FF000B0140008105000080800002058230000DA
:10500000C0140008000000000000000000F36F065C
:0400000508000105E9
:00000001FF
